:100000000C9477020C949F020C949F020C949F0214
:100010000C949F020C949F020C949F020C949F02DC
:100020000C949F020C949F020C9498270C946728C0
:100030000C94C6220C949F020C949F020C949F0275
:100040000C949F020C949F020C949F020C949F02AC
:100050000C949F020C9423230C949F020C949F02F7
:100060000C949F020C949F020C949F020C949F028C
:100070000C949F020C949F020C949F020C949F027C
:100080000C949F020C949F020C949F020C949F026C
:100090000C949F020C949F020C949F020C949F025C
:1000A0000C949F020C949F020C949F0250065006E1
:1000B0007C067C06E40602071A081A080D07A60744
:1000C000B707B707D428FB28F329FB28F3294729CA
:1000D0006A29F329C129D02914001A000800150043
:1000E000170000001C0018000C0012001300040090
:1000F0001600070009000A0000000B000D000E00AA
:100100000F0033001D001B00060019000500E00071
:100110001100100036003700380029002B00E300E2
:10012000E1002A00E2002C0001512D0034002800DB
:100130001E021F0252002F02300200004B0024005A
:100140002500260025022002500051004F00210208
:1001500000004E002100220023002E022F0030005C
:10016000260227022402E00035001E001F002000A6
:10017000310002534900E300E1002A00E2002C00B4
:100180000100370027002E0049004A0052004D00B0
:100190004B000000520040004100420043004C0070
:1001A000500051004F004E00000051003D003E0045
:1001B0003F0044000000A90000000000005CE000D7
:1001C00000003A003B003C0045000000AA00E300AC
:1001D000E1002A00E2002C001050460047004800D1
:1001E00000000000000000002A2B28000000000092
:1001F00000000000000000000000002900000000D6
:100200002C1E3420212224342627252E362D373843
:10021000271E1F202122232425263333362E37384C
:100220001F0405060708090A0B0C0D0E0F1011120A
:10023000131415161718191A1B1C1D2F3130232DD6
:10024000350405060708090A0B0C0D0E0F101112D4
:10025000131415161718191A1B1C1D2F3130354C85
:10026000000000000000000000000000000000008E
:10027000000000000000000000000000000000007E
:10028000000000007E0F00D4FFFFFFC700000078D1
:1002900041542B424C454849444D4F5553454255D6
:1002A00054544F4E3D0041542B424C454849444D17
:1002B0004F5553454D4F56453D25642C25642C25FF
:1002C000642C25640041542B424C45484944434F1B
:1002D0004E54524F4C4B45593D30782530347800C0
:1002E00041542B424C454B4559424F415244434F98
:1002F00044453D253032782D30302D253032782D53
:10030000253032782D253032782D253032782D2544
:100310003032782D253032780041542B47415047F8
:100320004554434F4E4E0041542B4556454E54457F
:100330004E41424C453D3078320041542B455645A4
:100340004E54454E41424C453D307831004F4B00B4
:100350004154453D300041542B4741504445564E91
:10036000414D453D4174726575730041542B424CBB
:1003700045484944454E3D310041542B4741504981
:100380004E54455256414C533D31302C33302C2C79
:100390000041545A0041542B424C45504F5745524E
:1003A0004C4556454C3D2D313200500379035603E0
:1003B0006B03950391030E03410074007200650006
:1003C00075007300000018035400650063006800A6
:1003D0006E006F006D0061006E0063007900000028
:1003E0000403090409023B00020100A0FA09040009
:1003F0000001030101000921110100012240000751
:10040000058103080001090401000103000000093F
:100410002111010001227B00070582032000011247
:10042000010002000000080912E5A1080001020015
:100430000105010902A10185020901A100050919AF
:10044000012908150025019508750181020501099A
:100450003009311581257F95027508810609381507
:1004600081257F950175088106050C0A38021581E2
:10047000257F950175088106C0C005010980A1018D
:10048000850319012AB700150126B70095017510DB
:100490008100C0050C0901A101850419012AA002EF
:1004A000150126A002950175108100C005010906FD
:1004B000A101050719E029E7150025019508750137
:1004C00081029501750881010507190029FF1500B2
:1004D00026FF009506750881000508190129059574
:1004E0000575019102950175039101C07E1E1124CD
:1004F0001FBECFEFDAE0DEBFCDBF11E0A0E0B1E07C
:10050000E6E1FCE502C005900D92A83AB107D9F7E3
:1005100024E0A8EAB1E001C01D92AD32B207E1F7D4
:1005200012E0C7E7D2E004C02197FE010E94412AF1
:10053000C637D107C9F70E941B140C94092E0C94DE
:1005400000009C013A9521153F4130F5BC0166271A
:100550007270AC01442754709C012227387094FFBC
:100560000FC090FF02C080E101C080E0672B09F05E
:100570008062452B09F08064232B79F08068089510
:10058000892F8170672B09F08260452B09F0846008
:10059000232B19F08860089580E00895CF93DF93AE
:1005A000EB010E94A102FE01DF91CF910994CF934C
:1005B000DF93EC01805E9109089710F0209719F401
:1005C00067E076E002C062E978E0CE010E94CE02E8
:1005D0008C2FDF91CF910C94D004CF93DF93EC015B
:1005E0000E947F05CE01805E9109089710F0209748
:1005F00019F46EE076E002C069E978E0CE01DF919F
:10060000CF910C94CE02CF93DF93EC010E94D702DE
:10061000C933D10549F42FEF83EF91E02150804099
:100620009040E1F700C00000CE01DF91CF910C9423
:10063000ED0281E0089581E008950C941B03089574
:100640000C941F031F93CF93DF9300D000D01F9211
:10065000CDB7DEB749835A836B833091AB01898173
:100660009A81311114C0662359F0222349F00E9467
:10067000650A182F682F89819A810E940E0A03C08B
:100680000E94390A182F69817A81812F04C00E9443
:10069000650A69817A810F900F900F900F900F90EB
:1006A000DF91CF911F910C949D11FC01262F408169
:1006B00051816281738184810C94220381E00895C9
:1006C000CF93DF93EC0160E00E945503BE01DF9100
:1006D000CF910C9420030C94CC120C94C812089562
:1006E0000E94B8080E946F032FE78AE196E021502C
:1006F00080409040E1F700C000000C9449230F9324
:100700001F93CF93DF938C0161E00E945503EC01AE
:10071000B8010E941D03882309F458C0B801CE0116
:100720000E947D17882309F451C0B801CE010E94B0
:10073000A220882309F44AC0B801CE010E949B1769
:10074000882309F443C0B801CE010E94FE1F88230C
:10075000E9F1F8018281882391F1CF3D8CE5D8073A
:1007600001F158F4CD3DFCE5DF07F1F0F8F4C115D7
:10077000DC4529F50E94700329C0CB35FDE5DF0774
:10078000C9F028F4CA32DD45D1F483E010C0CC357D
:10079000FDE5DF0791F0CD35DD4589F40E94E20EDD
:1007A0000EC00E94990F12C080E001C082E00E943A
:1007B000E4180CC00E94EB0E02C00E94EE0EC801AD
:1007C000DF91CF911F910F910C94190380E0DF917D
:1007D000CF911F910F9108950E9471040C94C32230
:1007E000DF92EF92FF920F931F93CF93DF93E82F47
:1007F000F0E0E052FE4FD490282F269526952695BE
:1008000030E0F901E058FD4F0491877010E0082EA8
:1008100002C0159507950A94E2F701701127F901B6
:10082000E059FD4FE490F12C082E02C0F594E794B6
:100830000A94E2F791E0E922FF24F901E05AFD4F22
:10084000C491D0E002C0D595C7958A95E2F7C170F2
:10085000DD270115110519F081EE0E94D004E11485
:10086000F10419F086EE0E94D0048D2D0E94FE0541
:10087000EF2819F086EE0E947F05012B19F081EE1A
:100880000E947F05CD2B51F08CE2DF91CF911F911B
:100890000F91FF90EF90DF900C94FE05DF91CF91C8
:1008A0001F910F91FF90EF90DF900895982F9F7008
:1008B0009A50963010F0805D01C0895A0C94F00374
:1008C00008950C94600481E008950C9463040895E5
:1008D000CF93C82F0E9461048C2F0E946504CF9192
:1008E00008950E9407220C9468040E9407229091A8
:1008F000AA01891721F08093AA010C946804089535
:10090000CF93DF93CDB7DEB72B970FB6F894DEBF4A
:100910000FBECDBF4F83588769877A878B87611158
:100920000E942E0E9E012F5F3F4F86E0F90111922B
:100930008A95E9F785E0FE013796D90101900D927D
:100940008A95E1F789819A814C815D81452B31F04F
:100950009F3F31F491E08F3F19F403C091E001C053
:1009600090E090FF09C049815A816B817C818D8123
:100970009E810E944C0D05C0C9010E945E03811139
:10098000F2CF2B960FB6F894DEBF0FBECDBFDF912E
:10099000CF910895FC01808191810E94A70A08955A
:1009A000CF93882309F4A9C0C82F8238C1F40E94CC
:1009B000072281FDA2C069E38091020190910301A9
:1009C0000E949D220E94500E2FEF80E792E021505E
:1009D00080409040E1F700C0000069E319C083380F
:1009E00001F50E94072280FD88C063E58091020125
:1009F000909103010E949D220E94500E2FEF80E7EC
:100A000092E0215080409040E1F700C0000063E593
:100A100080910201909103010E949F22CF910C943A
:100A2000500E8438C1F40E94072282FD66C067E43C
:100A300080910201909103010E949D220E94500E1C
:100A40002FEF80E792E0215080409040E1F700C016
:100A5000000067E4DDCF8CEF8C0F813AF8F48C2F27
:100A60000E94B51F811149C06C2F809102019091A5
:100A700003010E946722882349F06C2F80910201B4
:100A8000909103010E949F220E94500E6C2F809132
:100A90000201909103010E949D22C0CF80E28C0F41
:100AA000883048F4C77081E001C0880FCA95EAF722
:100AB0000E940E0EB3CFEBE5EC0FE33040F4F0E014
:100AC000E75BFE4F808190E0CF910C942F22E8E508
:100AD000EC0FE73150F4F0E0EE0FFF1FE55EFE4F44
:100AE00080819181CF910C944522CD3E30F08C2FA6
:100AF0000E94A014CF910C947215CF910895882371
:100B000009F464C0823879F40E94072281FF5EC034
:100B100069E380910201909103010E949D220E944D
:100B2000500E69E310C08338B1F40E94072280FFA1
:100B30004DC063E580910201909103010E949D22C6
:100B40000E94500E63E580910201909103010E9482
:100B50009F220C94500E843879F40E94072282FF61
:100B600035C067E480910201909103010E949D22AB
:100B70000E94500E67E4E7CF9CEF980F913A10F473
:100B8000682FE1CF90E2980F983050F4877091E091
:100B900001C0990F8A95EAF7892F0E94140ED9CFC8
:100BA0009BE5980F933020F480E090E00C942F2286
:100BB00098E5980F973120F480E090E00C9445225E
:100BC0008D3E20F00E94FB140C94721508951F9323
:100BD000CF93DF93182FEB010E94D004209741F0B0
:100BE0008FEC97E00197F1F700C000002197F6CF56
:100BF000812FDF91CF911F910C947F05893319F0DC
:100C000060E070E002C060E570E00C94E7058823C6
:100C100021F00E940E0E0C94500E0895882321F0AE
:100C20000E94140E0C94500E0895CF92DF92EF9212
:100C3000FF920F931F93CF93DF937C01D62FC72F83
:100C4000FC011281058102950F700E94040E882319
:100C5000B9F01123A9F08C2F807F803421F080E23D
:100C60008D0F883068F08091040482FD09C082E015
:100C70000E94B00E0E94040E91E0D82ED92601C029
:100C8000D12CCC2EC2948FE0C8228C2D90E08C30D9
:100C9000910508F0CFC1FC01EA5AFF4F0C94412A9C
:100CA0008C2F807FCF70882311F0C295C07F1123D5
:100CB00099F0CC2309F4AAC180E28D0F883010F09E
:100CC000D11104C08C2F0E940E0E03C08C2F0E94E5
:100CD000210E0E94500E9AC18D2F0E947F05CC23B9
:100CE00009F4A8C180E28D0F883038F1DD2329F1A5
:100CF0008C2F0E94270E24C08C2F807FCF708032D3
:100D000011F0C295C07FDD2319F0D130A1F13DC0B3
:100D10008091040482FF17C0112349F0CC2329F0ED
:100D20008C2F0E940E0E0E94500E80E070C180E059
:100D30000E947F05CC2309F47DC18C2F0E94140EE4
:100D40000E94500E77C1112371F0002341F0013051
:100D500031F40E94310E8C2B0E94390E6BC10E941F
:100D6000310E8C2B1DC0002319F0013009F462C133
:100D70000E94460E25C0112321F0063008F05AC10A
:100D80000EC0053008F056C11BC0112361F00023CE
:100D900031F0F701858180FF39C18F7085838C2FF9
:100DA0000E94070647C1002359F0D93309F03FC11B
:100DB000FFEF03EF11E0F15000401040E1F735C1C3
:100DC0008C2F0E940E0636C18C2F869586958370D7
:100DD00019F0813061F02EC1112321F08D2F9C2F4D
:100DE000937002C080E090E00E942F222BC111235B
:100DF00021F08D2F9C2F937002C080E090E00E9424
:100E0000452220C18D2F112319F00E94A01402C089
:100E10000E94FB140E94721515C18C2F837009F07B
:100E200047C011110BC12D2F229526952770220F37
:100E3000220F6D2F6F70862F90E0A0E0B0E0022EA1
:100E400004C0880F991FAA1FBB1F0A94D2F7D4FFB2
:100E500010C04FE050E060E070E004C0440F551F48
:100E6000661F771F2A95D2F740955095609570952B
:100E700003C040E050E0BA01C695C695C3708A0130
:100E80009B01082B192B2A2B3B2BC901B801C2301F
:100E900049F058F4C13019F00E942409CFC00E94D3
:100EA0001209CCC00E943609C9C00E941009C6C0F0
:100EB000112319F08C2F817001C08695882309F4C5
:100EC000BDC02D2F229526952770220F220F6D2F42
:100ED0006F70862F90E0A0E0B0E0022E04C0880F73
:100EE000991FAA1FBB1F0A94D2F7D4FF10C04FE06E
:100EF00050E060E070E004C0440F551F661F771F8C
:100F00002A95D2F7409550956095709503C040E0C2
:100F100050E0BA01C695C695C3708A019B01082BA3
:100F2000192B2A2B3B2BC901B801C23049F058F4C8
:100F3000C13019F00E94E90981C00E94D7097EC022
:100F40000E94FB097BC00E944A0978C0CF70112320
:100F500039F08C2F0E9470098D2F0E9407066EC0F9
:100F60008D2F0E940E068C2F0E94910967C0D23FE0
:100F700021F128F4D03F41F0D13FC1F043C0D33F2D
:100F800019F1D43F79F03EC0112341F0053008F04B
:100F900051C08C2F8F710E94B6094CC0063008F0EA
:100FA00049C0F7CF8091040482FF18C0112339F0A3
:100FB0008C2F8F710E9470093DC01123C9F38C2FB3
:100FC0008F710E94910936C0112329F08C2F8F71E7
:100FD0000E945B092FC00E9456092CC0112349F0C2
:100FE000CF718C2F0E94700963E08C2F0E94950EA8
:100FF00021C081E00E94B00E0230E0F082E00E9449
:10100000B00E18C0112331F0002391F28D2F0E94F1
:10101000D00410C0002399F2D93349F41FEF23EF15
:1010200031E0115020403040E1F700C000008D2F2A
:101030000E947F0588EF8C0D843020F40E940722E7
:101040000E946804DD20C9F00E94000E80FD15C0DA
:10105000F70112820E94FA0D0E947009C7010E94D6
:101060005E080E94FA0DDF91CF911F910F91FF90C2
:10107000EF90DF90CF900C949109DF91CF911F9169
:101080000F91FF90EF90DF90CF9008950F931F93F3
:10109000CF93DF93EC01688179818A810E94B20A43
:1010A0008C010E940D0A0E94FE08B801CE010E9428
:1010B0001506DF91CF911F910F910895CF93DF9384
:1010C000EC01988189812B813C81232B31F08F3F6A
:1010D00031F481E09F3F19F403C081E001C080E05A
:1010E00080FD1DC0CE010E947F03811110C00E94AF
:1010F000040E8823A1F08A81882389F0809104045A
:1011000082FD0DC082E0DF91CF910C94B00ECE0134
:101110000E944608CE01DF91CF910C946003DF91CD
:10112000CF910895882321F00E94210E0C94500E37
:101130000895882321F00E94270E0C94500E0895E4
:1011400080E090E00E942F2280E090E00E94452203
:101150000E942E0E0E94500E0E94A3160C9472152F
:1011600080910201909103010E94A1220C94A00899
:101170000E941E0E0C94B00892959F70963079F0E4
:1011800010F4925001C09A50923068F4803F69F098
:1011900018F4883E40F409C0843F29F406C0883E14
:1011A00020F0813F11F080E0089581E00895FC0176
:1011B000808191810E94A70A0E94BC080895CF9364
:1011C000DF9300D000D01F92CDB7DEB70F900F9005
:1011D0000F900F900F90DF91CF910895CF93DF93F1
:1011E00000D000D000D0CDB7DEB726960FB6F89469
:1011F000DEBF0FBECDBFDF91CF9108950895089552
:101200000C94FF080C9400090E9402096093CE011F
:101210007093CF018093D0019093D1010C94A008DA
:101220000C9404090F931F930091CE011091CF01EC
:101230002091D0013091D101602B712B822B932B07
:101240001F910F910C9404090F931F930091CE01ED
:101250001091CF012091D0013091D10160237123F1
:10126000822393231F910F910C9404090F931F93D2
:101270000091CE011091CF012091D0013091D10188
:1012800060277127822793271F910F910C940409DF
:101290000C94FF080E9448096093CA017093CB0127
:1012A0008093CC019093CD010C94A00860E070E095
:1012B000CB010C944A090F931F9341E050E060E08A
:1012C00070E08A019B0104C0000F111F221F331F11
:1012D0008A95D2F7C901B8011F910F910C944A0960
:1012E0000F931F9341E050E060E070E004C0440FB2
:1012F000551F661F771F8A95D2F78091CA0190917A
:10130000CB01A091CC01B091CD018A019B01082BAA
:10131000192B2A2B3B2BC901B8011F910F910C945B
:101320004A090F931F9341E050E060E070E004C071
:10133000440F551F661F771F8A95D2F74095509529
:10134000609570958091CA019091CB01A091CC01DC
:10135000B091CD018A019B01082319232A233B2345
:10136000C901B8011F910F910C944A090F931F9363
:1013700041E050E060E070E004C0440F551F661F7C
:10138000771F8A95D2F78091CA019091CB01A091E5
:10139000CC01B091CD018A019B01082719272A278A
:1013A0003B27C901B8011F910F910C944A090F9373
:1013B0001F930091CA011091CB012091CC01309173
:1013C000CD01602B712B822B932B1F910F910C94CD
:1013D0004A090F931F930091CA011091CB012091EC
:1013E000CC013091CD0160237123822393231F917F
:1013F0000F910C944A090F931F930091CA01109109
:10140000CB012091CC013091CD016027712782273B
:1014100093271F910F910C944A0908952BE0929FF6
:10142000800D1124E82FE695E695E695877051E04A
:1014300001C0550F8A95EAF785E0E89FF001112475
:10144000E455FE4F20E030E070E04081CB01022EF9
:1014500002C0969587950A94E2F78170819584275A
:101460008523842781932F5F3F4F2530310569F70E
:1014700008952BE0929F800D1124682F6695669544
:101480006695982F977085E0689FB001112440E021
:1014900050E080E0FB01E40FF51FE455FE4F208192
:1014A00030E0092E02C0369527950A94E2F72170A4
:1014B0003327042E01C0220F0A94EAF7822B4F5FD4
:1014C0005F4F4530510531F70895BF92CF92DF92BB
:1014D000EF92FF920F931F93CF93DF938C01C090F5
:1014E000CA01D090CB01E090CC01F090CD01809169
:1014F000CE019091CF01A091D001B091D101C82A25
:10150000D92AEA2AFB2ACFE1D0E0D701C6010C2E66
:1015100004C0B695A795979587950A94D2F780FD54
:1015200004C0219790F7B12C07C0BC2EB8018C2FB6
:101530000E94B0110197A9F38B2DDF91CF911F91DC
:101540000F91FF90EF90DF90CF90BF900895CF93D1
:10155000DF93EC010E94650ABE010E94B011DF9189
:10156000CF9108951F93CF93DF93EB019091AB013F
:10157000992321F0CB010E94A70A13C0882349F0C8
:10158000CB010E94650A182F682FCE010E940E0A17
:1015900004C0CB010E94390A182FBE01812F0E947E
:1015A000B011DF91CF911F9108951F93CF93DF93D7
:1015B000C091D20116E08091D301C81799F0D0E014
:1015C0001C9FF0011D9FF00D1124EC52FE4F408135
:1015D000518162817381848195810E94EE082196F8
:1015E000C770E9CFDF91CF911F9108954091040218
:1015F00050910502609106027091070280910802E5
:10160000909109020C94EE08EF92FF920F931F93B2
:10161000CF93DF938091090282958F7009F065C0A6
:1016200080910602882309F460C08091D201F09075
:10163000D30110910402009105026091070270919C
:10164000080291E01F3F09F090E0C0910001D091A5
:101650000101292F96E0E92E8F1509F446C0611586
:10166000710521F00F3F21F030E003C031E001C0EF
:10167000322F90E030FD36C0E89EF001E99EF00D7B
:101680001124DF01AC52BE4F11963C9111973013DB
:1016900029C03C91311326C012963C91129731110A
:1016A00021C013964D915C911497461B570B4C1714
:1016B0005D07C0F4809109028F70806180930902F8
:1016C000E752FE4F80818F708061808384E092E0DA
:1016D0000E945E08DF91CF911F910F91FF90EF90D4
:1016E0000C94D50A01968770B7CFDF91CF911F91E7
:1016F0000F91FF90EF9008959F92AF92BF92CF927B
:10170000DF92EF92FF920F931F93CF93DF93CDB7AA
:10171000DEB761970FB6F894DEBF0FBECDBF8C0168
:1017200085E0F801DE011D9601900D928A95E1F7A2
:10173000D8011296EC9090910402E091050220915C
:101740000702309108022115310531F0EF3F31F4E5
:1017500081E09F3F19F403C081E001C080E0B82F11
:10176000B1709B2E80FD47C1D8014C9111965C91C0
:1017700011971396AD90BC90149784E0C82E82E028
:10178000D82EF0900602B501621B730B2091000168
:1017900030910101FF2009F4D9C08091090262173C
:1017A000730708F095C0282F207F09F052C05E1300
:1017B00013C0491311C0FE2CE1100EC08F70806160
:1017C000809309020E94F60AC6010E945E08809179
:1017D0000902F80185834DC1AB2831F05F3F31F438
:1017E00081E04F3F19F403C081E001C080E080FD3B
:1017F00003C081E08E2502C080E090E0F82FF170F8
:10180000FF2E80FF1CC08091D2012091D30136E0D1
:10181000821709F40BC190E0389FF001399FF00D59
:101820001124EC52FE4F6181561306C060814613AD
:1018300003C06281E61203C001968770E9CFFE2CD7
:10184000EE2009F416C1809109028160809309029B
:1018500054C05E1306C0491304C0E11002C0F80171
:1018600099C0C8010E94D708882361F1EE2051F188
:1018700020910902822F82958F7090E0029774F078
:10188000809104029091050298878F831986BB8608
:10189000AA862C87CE0107960E945E0886E0F80192
:1018A000A4E0B2E001900D928A95E1F70E94040B4A
:1018B0000E94F60A0AC05E1711F1C8010E94D708FB
:1018C00081112CC0C8010E945E08FF24F394D1C08E
:1018D000282F207F81F77A2DB98AA88A6E2D8989D1
:1018E0000E94DF0884E092E00E945E0886E0D60154
:1018F0001D928A95E9F70E94F60AF12CBAC04913A5
:10190000DCCFE110DACFF8018583C8010E945E08C0
:1019100086E0D6011D928A95E9F7ABC0EE2091F2E0
:1019200020910902822F82958F7090E002970CF42B
:10193000B5CF80910402909105029A8389831B821E
:10194000BD82AC822E83CE010196A6CF62177307AB
:1019500008F044C0FE2CEE2009F4B4CF5E1330C072
:1019600049132EC02091090220FD21C0822F8295AB
:101970008F70482F50E041155105C9F0F8012583BB
:101980004F30510541F08F5F982F9295907F822FB5
:101990008F70892B8583C8010E945E0886E0F8015C
:1019A000A4E0B2E001900D928A95E1F73CC086E098
:1019B000F801A4E0B2E001900D928A95E1F759C0D8
:1019C000C8010E94D708811169CF80910902816006
:1019D00080930902C8010E945E084BC07A2DB98A23
:1019E000A88A6E2D89890E94DF0886E0D6011D92A3
:1019F0008A95E9F718C0EE2009F464CFC8010E9467
:101A0000D708F82E882309F45DCF86E0F801A4E01A
:101A1000B2E001900D928A95E1F784E092E00E9495
:101A2000CA040E94040B0E94F60A23C04D875E87F9
:101A30008D859E850E94A70A292F22952F7022301E
:101A400028F49F7039F0811105C00BC0243028F4B0
:101A50009F7049F4805E883020F0C8010E945E08C3
:101A60009F2CF92C06C0D80115969C91907F91F778
:101A7000F8CF8F2D61960FB6F894DEBF0FBECDBFA5
:101A8000DF91CF911F910F91FF90EF90DF90CF905A
:101A9000BF90AF909F9008951F93CF93DF93CDB7E2
:101AA000DEB72C970FB6F894DEBF0FBECDBF4F83C5
:101AB000588769877A878B879C87CE0107960E9413
:101AC0007C0B8823D1F09F8188852A853B85232B39
:101AD00031F08F3F31F481E09F3F19F403C081E082
:101AE00001C080E080FD47C04F81588569857A85B7
:101AF0008B859C850E94EE083EC086E0FE013796ED
:101B0000DE01119601900D928A95E1F7FF81E8853B
:101B10006A857B856115710531F0EF3F31F481E015
:101B2000FF3F19F403C081E001C080E080FD23C0C5
:101B30002091D30130E0C901019687709927409127
:101B4000D20150E084179507F1F1F983EA837D8390
:101B50006C8396E0929FD001939FB00D1124AC52FC
:101B6000BE4FFE01319601900D929A95E1F7809358
:101B7000D3010E94D50A16E08091D2019091D30141
:101B8000891771F1189FC00111248C529E4F0E9439
:101B90007C0B882329F1E091D2011E9FF0011124D2
:101BA000EC52FE4F40815181628173818481958125
:101BB0000E94EE088091D20190E0019687709927EB
:101BC0008093D201D9CF0E94B8081092D30110920D
:101BD000D201E4E0F2E086E0DF011D928A95E9F7A8
:101BE0002C960FB6F894DEBF0FBECDBFDF91CF911C
:101BF0001F91089580911202859585958595089588
:101C0000809112028770089590911202977081E07E
:101C100009F480E0089580911D02089590911D02BD
:101C2000892B80931D020895809590911D02892330
:101C300080931D02089580931D02089510921D0245
:101C4000089590911C02892B80931C020895809521
:101C500090911C02892380931C02089510921C020B
:101C6000089580911302089508950C94340E0C94F5
:101C7000350E9091040492FD08C0909113029817BC
:101C800021F0809313020C94370E08958091130273
:101C9000882329F01092130280E00C94370E0895E7
:101CA000CF93DF93E0910201F091030180911D0237
:101CB0008083E0910201F0910301908180911C02E8
:101CC000892B808380911302882381F0E0910201A7
:101CD000F09103019081892B808380910201909182
:101CE00003010E945B2281110E94460EC0910201F5
:101CF000D091030148E050E06AE072E0CE010E941A
:101D00009B2A892B69F088E0FE01AAE0B2E00190ED
:101D10000D928A95E1F7CE01DF91CF910C941622B6
:101D2000DF91CF9108950C94340E9091040492FDAC
:101D300010C098E0899F90011124262B2093120255
:101D40000E947009809112028595859585950C9465
:101D5000930E0C9470091092120280E00C94930E72
:101D6000209112028095822380931202982F9770FF
:101D700099F430E0482F082E000C550B2417350736
:101D800059F09091040492FD07C08595859585953D
:101D90000E9491090C94AB0E08959091040492FB5B
:101DA000222720F9281769F080FB92F99093040408
:101DB00080910304909104040E94150F82E00C941A
:101DC000B00E08958091040482FB882780F991E089
:101DD00089270C94CD0E81E00C94CD0E80E00C94FC
:101DE000CD0E80E090E00E94982D21E0893E9E4F2C
:101DF00009F020E0822F089582E090E00C94902D6D
:101E000083E090E00C94902DCF9384E090E00E94CA
:101E1000902DC82F82E290E00E94902D2C2F30E070
:101E2000A901582BCA01CF910895CF93C92F682FCC
:101E300084E090E00E949E2D6C2F82E290E0CF9192
:101E40000C949E2DAB01BC018FE090E00C94B02D62
:101E5000AB01BC0183E190E00C94B02D60E070E038
:101E6000CB010C94280F60E070E0CB010E94220FA0
:101E70000C942E0F69EE7EEF80E090E00E94BC2D66
:101E800060E082E090E00E949E2D60E083E090E0C0
:101E90000E949E2D1092CE011092CF011092D0017F
:101EA0001092D10160E084E090E00E949E2D60E0FD
:101EB00082E290E00E949E2D60E085E090E00E942A
:101EC0009E2D60E086E090E00E949E2D6FEF87E0FF
:101ED00090E00E949E2D40E050E0BA0188E090E042
:101EE0000E94B02D60E08DE090E00E949E2D40E0C9
:101EF00050E0BA0188E190E00E94B02D60E087E1F7
:101F000090E00E949E2D40E050E0BA018CE190E00C
:101F10000E94B02D60E070E080E290E00E94BC2D55
:101F200040E050E0BA0188E190E00E94B02D0C94AE
:101F3000330F0C943A0F682F8EE090E00C949E2D96
:101F40000E94082360932A0270932B0280932C0234
:101F500090932D02609326027093270280932802AB
:101F600090932902089585B7806885BF85B78068FA
:101F700085BF089581E008950C94BA0F08950C94DC
:101F8000BE0F0C94BE0F0C94C10F0C94BE0F0C949A
:101F9000C50F0C94BE0F0E94B30F8CE892E10E9413
:101FA000FD210E94C90F0C94C70F0E94BF0F0C9413
:101FB000BE0F0E948F120E9467040E94D91680E013
:101FC0000C94E4180E94F3220E9474130E94D90F0B
:101FD0000C94C30F5F926F927F928F929F92AF92F9
:101FE000BF92CF92DF92EF92FF920F931F93CF9306
:101FF000DF93CDB7DEB72A970FB6F894DEBF0FBEDA
:10200000CDBF0E948913C82E81110E94A00F3EE10E
:10201000832E32E0932E00E010E0502E802F0E949D
:10202000B3125C01F401619071904F01682679262A
:1020300061147104B1F40F5F1F4F0430110569F78B
:102040008FEF89838A831B820E94FC228160782F14
:102050009D838C8349815A816B818D810E9480048C
:102060003AC080912E0281FD0E94BC12D12CEE2438
:10207000E394F12CC3018E219F21892B29F10E9429
:10208000BC0F8823A9F0DE825F82AE20BF2081E0F2
:10209000AB2809F480E088870E94FC228160782FB9
:1020A0009A8789874E815F8168858A850E9480042E
:1020B000000F111FF801E25EFD4F80819181E8263B
:1020C000F926F182E08207C0D394EE0CFF1CFBE0FE
:1020D000DF12D0CFB0CF81E0C11001C080E02A96DE
:1020E0000FB6F894DEBF0FBECDBFDF91CF911F9129
:1020F0000F91FF90EF90DF90CF90BF90AF909F90A7
:102100008F907F906F905F9008950E94EA0F0E94D9
:1021100090150C947504CF93DF930E94B511EC01D8
:10212000811521E5920708F045C0811530E5930738
:1021300008F094C0883E910528F5803E910508F08E
:10214000F8C0883A910570F4853A910508F07CC092
:102150008130910509F475C008F4E8C0049708F0CF
:10216000E8C0E4C08F3B910508F0E0C0C85AD0E059
:10217000CC0FDD1FC45BDE4F0990D881C02DCE018E
:102180009464D8C0811540E2940758F4811551E059
:10219000950708F0CEC08D3E910508F4C7C0906544
:1021A000C9C0C11580E4D80708F4C0C0DF70CE01F3
:1021B000906AC0C0811525E59207A8F4811534E521
:1021C000930708F095C0811543E5940708F07BC09C
:1021D000811552E5950708F061C0D82FCC27CE01B4
:1021E000816F906AA7C0C11589E5D807A0F4C11511
:1021F00028E5D20708F082C0C11536E5D30708F0FC
:1022000095C08C2F0E9449128F7190E0D82FCC2757
:10221000CE0190628FC0C1154AE5D40708F474C09E
:10222000CE0190568115904208F080C08D2F8F719D
:102230000E944912DD27D0628F71AE01582BCA016E
:1022400079C081E090E076C0C55AD0E0C658DE4F34
:102250008881C82FD0E0CE0190646CC074E0969560
:1022600087957A95E1F7282F23703C2F337081E012
:1022700090E002C0880F991F3A95E2F79C68AC0184
:10228000522B9A019C2F9F709695969550E2959FA0
:10229000E0011124C9018C2B9D2B4CC08370992720
:1022A00021E030E002C0220F331F8A95E2F79C2F15
:1022B0009695969580E2989FE0011124C22BD32B2E
:1022C000CE019C6837C08370992721E030E002C0BE
:1022D000220F331F8A95E2F79C2F9695969540E240
:1022E000949FE0011124C22BD32BCE019A6822C007
:1022F000D82FCC27CE01846F906A1CC0DC2FCC274E
:10230000CE01806F906A16C08C2F8F700E94491288
:1023100094E0D695C7959A95E1F7CF70D0E0DC2F81
:10232000CC27D0699E01282BC90104C080E090E031
:1023300001C0CE01DF91CF9108952CE2829FC001B0
:102340001124FC012BE0729FE00DF11D1124E60F1A
:10235000F11DEE0FFF1FE852FF4F859194910895F4
:102360000E949D110E948B1008958238910569F199
:10237000B0F48133910509F46DC048F489329105B8
:1023800009F463C08A32910509F469C00895853360
:10239000910509F455C089339105B9F00895833E3C
:1023A000910569F138F4803E9105B1F0823E9105C6
:1023B00009F10895863E9105A9F1873E9105B9F18D
:1023C000843E910509F064C023C02091030420FDE0
:1023D0004FC021FD4DC008958091030480FD44C08D
:1023E0008091040480FF44C08091030484FD42C0B6
:1023F00083EE4DC08091030482FF38C0F5CF8091F9
:10240000030482FD33C08091040480FD31C0ECCF11
:102410008091040481FF32C08091030484FD2AC0AE
:1024200087EE35C08091030483FF26C0F5CF8091ED
:10243000030483FD21C08091040481FD1FC0ECCF03
:102440008091030485FD1CC01DC08091030485FD9F
:1024500019C016C08091030486FD16C017C0809174
:10246000030486FD13C010C089E311C082EE0FC0C3
:1024700080EE0DC080E00BC086EE09C084EE07C080
:1024800089E205C085E303C08AE201C081E390E0F0
:1024900008959091030492FF0DC0282F28712830D1
:1024A00019F4877F846006C0282F2471243011F42A
:1024B0008B7F886093FF0DC0282F2871283119F475
:1024C000877E846106C0282F2471243111F48B7E0D
:1024D00088612091040420FF0DC0382F38713830F6
:1024E00019F4877F816006C0382F3171313011F4C3
:1024F0008E7F886021FF0DC0282F2871283119F4A4
:10250000877E816106C0282F2171213111F48E7ED2
:10251000886194FD877E089580E0089508950E9463
:10252000F10E811102C00E94990F0E94FC0E80934F
:102530002E020E94040F90930404809303040E94CF
:102540008E120E94000F682F70E080E090E00E94E1
:1025500010096091CA017091CB018091CC019091DA
:10256000CD010C944809E82FF0E0EE0FFF1FE35F68
:10257000FB4F808191810895089580E58A95F1F758
:10258000089500C008950C94BD1208950C94C512CE
:102590000C94C6120C94C5120C94CA12F894E82F2D
:1025A000E295EF70F0E031A1282F2F7081E090E0EC
:1025B00001C0880F2A95EAF7982F9095932391A34D
:1025C00092A1892B82A3789408950F931F93CF93A0
:1025D000DF93C8E8D1E089918F3F11F00E94CE12BD
:1025E00081E0CC38D807B9F7CDE7D1E008E811E0B1
:1025F00089918F3F11F00E94CE120C171D07C1F771
:10260000DF91CF911F910F910895BF92CF92DF92EA
:10261000EF92FF920F931F93CF93DF938C01C62FFE
:10262000D0E0CE0188579E4F6C01FC0190819F3F06
:1026300009F450C0B62EF894E92FE295EF70F0E05F
:1026400081A19F7021E030E001C0220F9A95EAF746
:10265000822B81A382A12095282322A378940E9413
:10266000C112EDE7F1E048E851E021E030E0E12C73
:10267000F12C61916F3F89F0A62FA295AF70B0E069
:1026800090968C9190E06F7002C0959587956A95B1
:10269000E2F780FD02C0C90102C080E090E0E82AB4
:1026A000F92A220F331F4E175F0719F7F6018081B1
:1026B0008F3F11F00E94CE1261E0E114F10409F4A1
:1026C00060E08B2D0E94C312CC0FDD1FC00FD11F05
:1026D000F982E882DF91CF911F910F91FF90EF90E7
:1026E000DF90CF90BF9008950E94E51288E0EDE062
:1026F000F4E0DF01982F1D929A95E9F7E5E0F4E008
:10270000DF011D928A95E9F784E00E94D4130C94AE
:102710006B03FF920F931F93CF93DF93CDB7DEB779
:1027200028970FB6F894DEBF0FBECDBF8E010F5FA6
:102730001F4F88E0F80111928A95E9F7F12C6F2D6F
:10274000C8010E940513F394F4E0FF12F8CF48E0AB
:1027500050E0B80185E094E00E949B2AFF24F394A6
:10276000009709F4F12C892B41F088E0F801A5E0ED
:10277000B4E001900D928A95E1F72F2D44E06DE0D1
:1027800074E085E094E00E94D5130E946D038F2DC4
:1027900028960FB6F894DEBF0FBECDBFDF91CF9164
:1027A0001F910F91FF9008950895FF920F931F932B
:1027B000CF93DF93F82E092F162FD72FC42F222364
:1027C00049F081E0809331020E94FC229093300214
:1027D00080932F02809131028823D9F080912F02BB
:1027E000909130020E941423059798F0EF2DF02F5E
:1027F000A12FBD2F80E090E04C2F50E0841795076B
:1028000034F4219131912D933D930196F7CF10929D
:102810003102DF91CF911F910F91FF9008950E9497
:102820001E250E94E20F0C942A250E942E250E944C
:1028300085100C942F250E94C5220E9405250E9418
:10284000CB0F0E940F140E9415140E94D50FFBCFCE
:102850008091380280FF06C06091090170E0660F28
:10286000771F26C081FF04C06091090184E005C084
:1028700082FF07C06091090188E0689FB0011124C0
:1028800017C0909137029923D1F0609108019617F3
:1028900088F72091090188E0289F90011124929FD8
:1028A000A001939F500D112470E0CA010E942D2AAF
:1028B0006038710540F46115710519F406C068E0CF
:1028C00070E0862F08958FE7089581E00895809144
:1028D000380280FF08C06091050170E0759567952A
:1028E0007595679521C081FF06C06091050170E074
:1028F0007595679519C082FF04C06091050170E06D
:1029000010C090913602992399F0609104019617B6
:10291000A0F780910501899FC001112470E00E94F9
:102920002D2A6038710540F46115710519F406C04F
:1029300061E070E0862F08958FE7089581E00895A3
:102940008D3E21F40E942814819504C08E3E29F406
:102950000E94281480933C0208958F3E21F40E9427
:102960002814819504C0803F29F40E942814809384
:102970003B020895893F19F40E94671405C08A3FFD
:1029800031F40E946714819580933D0208958B3F36
:1029900021F40E946714819504C08C3F29F40E94A1
:1029A000671480933E0208959FE0980F983078F462
:1029B00021E030E0A90102C0440F551F9A95E2F7CB
:1029C000CA0190913A02892B80933A0208958D3F73
:1029D00021F48091380281600BC08E3F21F48091F8
:1029E0003802826005C08F3F29F4809138028460EC
:1029F0008093380208958D3E39F490913C0297FF00
:102A000035C010923C0259C08E3E29F490913C0290
:102A10001916BCF32BC090913B028F3E29F497FF0F
:102A200025C010923B0249C0803F19F41916CCF31F
:102A30001DC090913D02893F29F41916BCF41092F3
:102A40003D023BC08A3F19F497FF10C0F8CF8B3F7F
:102A500039F490913E0297FF09C010923E022DC0BA
:102A60008C3F21F490913E021916BCF39FE0980F21
:102A7000983080F421E030E0A90102C0440F551FD6
:102A80009A95E2F7CA01809590913A028923809342
:102A90003A0213C08D3F21F4809138028E7F0BC023
:102AA0008E3F21F4809138028D7F05C08F3F29F43D
:102AB000809138028B7F8093380280913B02811194
:102AC00006C080913C02811102C0109237028091B1
:102AD0003D02811106C080913E02811102C0109218
:102AE000360208950E94FC2220913B02211104C06D
:102AF00020913C02222321F09093350280933402EE
:102B000020913D02211104C020913E02222321F098
:102B1000909333028093320289E392E00C94212255
:102B2000EF92FF920F931F93CF93DF9300D000D0CB
:102B300000D0CDB7DEB786E0E9E3F2E0DE01119622
:102B400001900D928A95E1F7E0903B02F0903C02F3
:102B500000913D0210913E0210923B0210923C0205
:102B600010923D0210923E02E11003C0FF2009F4D2
:102B70005DC080913402909135020E941423AC0113
:102B800090913702992339F020910A0130E02417FF
:102B9000350758F04BC020910B018AE0289F900127
:102BA00011242417350718F041C09F3F19F09F5F8B
:102BB00090933702EE2061F00E9428141E1414F046
:102BC0009FEF01C091E0989F902D112490933B02BC
:102BD000FF2061F00E9428141F1414F09FEF01C021
:102BE00091E0989F902D112490933C0230913B02EC
:102BF0003323E1F020913C022223C1F045EB340362
:102C0000C0011124992319F090933B0203C081E085
:102C100080933B0235EB2303C0011124992319F063
:102C200090933C0203C081E080933C02011103C0F9
:102C3000112309F45DC080913202909133020E9409
:102C40001423AC0190913602992339F020910601AA
:102C500030E02417350758F04BC0209107018AE077
:102C6000289F900111242417350718F041C09F3F79
:102C700019F09F5F90933602002361F00E94671461
:102C8000101614F09FEF01C091E0989F902D112431
:102C900090933D02112361F00E946714111614F005
:102CA0009FEF01C091E0989F902D112490933E02D8
:102CB00030913D023323E1F020913E022223C1F006
:102CC00045EB3403C0011124992319F090933D0280
:102CD00003C081E080933D0235EB2303C001112442
:102CE000992319F090933E0203C081E080933E0245
:102CF00080913B0281110BC080913C02811107C081
:102D000080913D02811103C080913E0281110E9499
:102D10007215EB82FC820D831E8386E0FE013196E4
:102D2000A9E3B2E001900D928A95E1F726960FB6DD
:102D3000F894DEBF0FBECDBFDF91CF911F910F91F1
:102D4000FF90EF900895E9E3F2E086E0DF011D9245
:102D50008A95E9F7109237021092360210923802E3
:102D60000895CF93DF9397FF0DC0FB0122812223AB
:102D700049F0EC010E94EF16CE019F770E94621786
:102D80000E943C1781E0DF91CF9108959091160445
:102D9000923069F48A3040F490E009966AE070E07D
:102DA0000E942D2A875A01C086500C94FE050C946F
:102DB00056048CE090E00E94902D90E0A0E0B0E0FE
:102DC0008093160490931704A0931804B0931904E9
:102DD0000895609116048CE090E00C949E2D0E9462
:102DE00013228695817080931B040E9413228170A8
:102DF0008093150480911604813039F480911B046E
:102E0000882319F089E30E94FE050E940B0E80932F
:102E10001A040E941E0E80911604813071F048F051
:102E2000823081F0843009F586EE0E94FE0588E14B
:102E30001AC082EE0E94D00418C088E193E00E947C
:102E4000030313C080911504811103C083E50E9420
:102E5000FE0582EE0E94D0048FE19EE40197F1F717
:102E600000C0000087E50E94FE058FE19EE4019707
:102E7000F1F700C00000089580911604813059F0E8
:102E800030F0823089F08430C9F488E215C082EED7
:102E90000E947F0513C08CE20E94FE0580911B04F6
:102EA000882361F089E308C082EE0E947F0580914B
:102EB0001504811103C083E50E94FE0580911A0468
:102EC0000C941B0E0F931F93CF93DF938C01CCE0D8
:102ED000D0E0C8010C2E02C0969587950A94E2F7BF
:102EE0008F700E94C6162497CC3F8FEFD80789F7C2
:102EF000DF91CF911F910F9108950F931F93CF935F
:102F0000DF93EC018B01FB018281882361F00E9439
:102F10000B0ECE01825E9C458530910520F4809396
:102F200016040E94E916B801CE01DF91CF911F91DE
:102F30000F910C94B116CF93DF93EC01FB018281CA
:102F4000882309F43CC1C430FDE5DF0760F4CB3FC2
:102F50009CE5D90788F49E0122503C452431310577
:102F600008F02EC109C0C236EDE5DE0729F0C63AE9
:102F7000FDE5DF0709F024C10E94040F90930404CB
:102F800080930304C1318CE5D80709F4C6C008F06A
:102F900042C0C930ECE5DE0709F49BC000F5C5303E
:102FA0008CE5D80709F485C078F4C330ECE5DE077A
:102FB00009F478C008F07AC0C230DC4509F0F5C0E9
:102FC000809103048160EFC0C7309CE5D90709F404
:102FD00078C008F07AC0809103048061E4C0CD30ED
:102FE000FCE5DF0709F487C058F4CB309CE5D9072E
:102FF00009F479C008F07BC08091030488606FC039
:10300000CF30FCE5DF0709F480C008F082C0809172
:103010000304877FC8C0CE3F9CE5D90709F471C07F
:1030200000F5C531FCE5DF0709F485C068F4C3315C
:103030009CE5D90709F475C008F095C00E94B8084E
:10304000809103048F77AFC0CC3FFCE5DF07A9F187
:1030500008F054C0CB3FDC4509F0A7C080910404C0
:1030600040C0C230EDE5DE0709F489C058F4C1154F
:103070008DE5D80709F45AC008F069C080910404AE
:1030800082602FC0C236EDE5DE0709F47CC0C63A87
:10309000FDE5DF0709F481C0C330DD4509F085C0D7
:1030A00080E06EC08091030482607DC08091030443
:1030B00016C080910304886076C080910404826009
:1030C0004FC08091030480626EC0809103048064CD
:1030D0006AC00E94B80880910304806864C084605C
:1030E00062C081603DC0809103048E7F5CC080918E
:1030F00003048D7F58C08091030416C0809104049E
:1031000018C0809104048D7F2BC0809103048F7EB2
:103110004AC0809103048F7D46C0809103048F7B59
:1031200042C080910304877F8B7F3DC0809104045F
:103130008D7F8E7F15C08091030482FB222720F9AA
:1031400091E0922790FB82F990FB83F92CC080914B
:103150000404982F909591708E7F892B90FB81F9B4
:103160008093040422C00E94B8088091030487FB66
:10317000222720F991E0922790FB87F914C081E083
:103180000E949B0F12C08091030484FB222720F928
:1031900091E0922790FB84F906C080910304982F58
:1031A000909590FB80F980930304809103049091A3
:1031B00004040E94150F0E94B80880E001C081E05D
:1031C000DF91CF9108950895CF93C82F0E94E318FF
:1031D000C0933F02CF9108950E94272A811104C015
:1031E0000E94AE1C83E0089582E0089580913F0222
:1031F000811102C00C94EC180895873941F178F4DC
:10320000863349F130F4843321F1853331F584E29A
:1032100008958439D1F0863901F581E20895843F1B
:1032200071F030F4803FD9F0813FB9F481E0089526
:10323000863F49F030F0873F81F487E0089584E0CD
:10324000089585E0089586E0089580E2089582E279
:10325000089583E2089585E208958FE1089580E05E
:10326000089595E890937A00982F907290689093C3
:103270007B008F7190910C01892B80937C00809151
:103280007A00806480937A0080917A0086FDFCCF7A
:10329000809178002091790090917A009F779093A7
:1032A0007A0090E0922B08950E94FD180C94311939
:1032B000EF92FF920F931F93CF93DF93EC018B015B
:1032C00022E030E040E060E084E30E94FC200E94C5
:1032D000FC227C0188810E9475218E3F9105A9F412
:1032E0000E94D52182E48A95F1F700C022E030E007
:1032F00040E060E084E30E94FC20C7010E941423A8
:103300008017910738F3C0E00AC06B816F7770E0D7
:103310006D5F7F4FCE0101960E94A521C1E00E9402
:10332000D5218C2FDF91CF911F910F91FF90EF90BE
:103330000895EF92FF920F931F93CF93DF93EC01C9
:103340007B010E94FC228C0166990CC082E08A9568
:10335000F1F700C0C8010E9414238E159F05A0F349
:10336000C0E035C022E030E040E060E084E30E944D
:10337000FC200E948D2188838E5F8230A8F40E94F9
:10338000D52182E48A95F1F700C022E030E040E0E8
:1033900060E084E30E94FC20C8010E9414238E1583
:1033A0009F0538F3C0E011C063E070E0CE010196E4
:1033B0000E94BD216B816F7770E06131710524F44B
:1033C000CE0104960E94BD21C1E00E94D5218C2F20
:1033D000DF91CF911F910F91FF90EF9008951F9370
:1033E000CF93DF93CDB7DEB764970FB6F894DEBF07
:1033F0000FBECDBFE091450290914402E91709F458
:103400003FC0182F669B21C066E970E0CE0101968F
:103410000E9499198823A1F18C8187FD0DC020910C
:10342000450280914402281759F130E02F5F3F4F49
:103430002170332720934502112311F19091450209
:103440008091440298131AC01BC0F0E0EE0FFF1FDA
:10345000E05CFD4F808191810E9414238D32914068
:1034600078F08091450290914402891749F090E0EC
:103470000196817099278093450202C06699C4CF56
:1034800064960FB6F894DEBF0FBECDBFDF91CF912B
:103490001F9108956F927F928F929F92AF92BF92E9
:1034A000CF92DF92EF92FF920F931F93CF93DF9310
:1034B000CDB7DEB7A8970FB6F894DEBF0FBECDBF6D
:1034C0007C018B016A014901FC0101900020E9F7B0
:1034D000CF0101975C01672B61F0909144028091CC
:1034E0004502981721F081E00E94EF19F6CFF8010C
:1034F000108240E1742E5AE0652EA5014E195F0935
:10350000888D41315105DCF07D8A1E8A6F8A807872
:1035100080618068888FF701DE015996872D0190C0
:103520000D928A95E1F7B401CE0145960E94581993
:10353000882309F464C0F0E1EF0EF11CDECF80E1D6
:103540008D8B1E8A8AE08F8B842F8F77888F5527EB
:10355000B701CE0149960E94A82AB401CE01459632
:103560000E945819F82E882309F449C00115110545
:10357000E1F40E94FC228C018091440290E09C01C5
:103580002F5F3F4F2170332740914502421709F4C6
:103590005AC0880F991FFC01E05CFD4F1183008326
:1035A000209344020E94FC2252C05801AC0CBD1C66
:1035B00078016CE271E0CE0101960E94991988238E
:1035C000F1F08981803219F0F801108218C08C81E5
:1035D0008F77CA2CCE188C1508F4C82ECC2051F049
:1035E000D12CA601BE016B5F7F4FC7010E94A82AA4
:1035F000EC0CFD1C8C8187FDDCCFF70106C0F12CA3
:1036000026C07F0180818A3039F41082F70131971A
:103610000E171F07B0F302C08D30B9F36AE070E0F7
:10362000C8010E94BC2A009719F08C010F5F1F4F40
:103630006DE473E0C8010E94822A21E0892B09F021
:1036400020E0F22E04C080E00E94EF1995CF8F2D6C
:10365000A8960FB6F894DEBF0FBECDBFDF91CF9115
:103660001F910F91FF90EF90DF90CF90BF90AF90A0
:103670009F908F907F906F9008958F929F92AF92BE
:10368000BF92CF92DF92EF92FF920F931F93CF934F
:10369000DF93CDB7DEB77C015B014A01CDB6DEB664
:1036A0000E94922A01962DB73EB7281B390B0FB600
:1036B000F8943EBF0FBE2DBF0DB71EB70F5F1F4F53
:1036C000B701C8010E948B2A26E930E0A401B501A8
:1036D000C8010E944A1A0FB6F894DEBE0FBECDBED6
:1036E000DF91CF911F910F91FF90EF90DF90CF90DE
:1036F000BF90AF909F908F9008958F929F92AF92BE
:10370000BF92CF92DF92EF92FF920F931F93CF93CE
:10371000DF93CDB7DEB7CA57D1090FB6F894DEBF35
:103720000FBECDBF7C019091440280914502981359
:1037300001C19091D7038091D603981709F4FAC07C
:103740008AE0899F900111242A5B3D4FF901DE0137
:10375000AF58BF4F01900D928A95E1F7F901C080F3
:1037600015810681D780908481840E94FC229093E9
:10377000E3038093E203F1E0CF1679F1CF1628F04E
:1037800022E0C21609F452C0BAC060EE72E0CE0167
:1037900001965C010E948B2A1F928F921F929F922A
:1037A0001F92DF921F920F931F921F93E6968FAD89
:1037B000E6971F928F93E5968FADE5971F928F93B3
:1037C000BF92AF921F9280E38F938E010F5B1F4FCA
:1037D0001F930F930E94CF2A1BC065EC72E08E01ED
:1037E0000F5F1F4FC8010E948B2AE6968FADE697A8
:1037F0008F93E5968FADE5978F931F930F931F924D
:1038000080E38F93005C1F4F1F930F930E94CF2A7A
:10381000970140E050E060E070E0C8010E944A1A61
:103820000FB6F894DEBF0FBECDBF67C066EA72E088
:10383000CE0101965C010E948B2A802F002E000C85
:10384000990B9F930F93812F012E000C990B9F933F
:103850001F93E6968FADE697282F082E000C330BAA
:103860003F938F93E5968FADE597282F082E000C98
:10387000330B3F938F93BF92AF921F9280E38F934E
:103880008E010F5B1F4F1F930F930E94CF2A97014A
:1038900040E050E060E070E0C8010E944A1A0FB6B4
:1038A000F894DEBF0FBECDBF8823C1F160E972E09E
:1038B000C8010E948B2AD0FE05C06CE871E0C801E7
:1038C0000E94B12AD1FE05C06EE871E0C8010E94D5
:1038D000B12AD2FE03C060E971E004C0D11005C076
:1038E00062E971E0C8010E94B12A970140E050E00E
:1038F00060E070E0C8010E944A1A882379F0809144
:10390000D7039091D6038917A9F090E0019668E259
:1039100070E00E942D2A8093D7030CC0FFE729EAAC
:1039200033E0F15020403040E1F700C0000081E07A
:103930000E94EF19C658DF4F0FB6F894DEBF0FBED6
:10394000CDBFDF91CF911F910F91FF90EF90DF904E
:10395000CF90BF90AF909F908F9008958091D803A3
:1039600008950F931F93CF93DF93CDB7DEB7C2585F
:10397000D1090FB6F894DEBF0FBECDBF8091D90339
:1039800081111EC01092DA031092D8036E987698B7
:103990000E94F420549A5C9A5C988FE19EE401970F
:1039A000F1F700C000005C9A9FEF29E688E1915092
:1039B00020408040E1F700C0000081E08093D903FF
:1039C0001092DA030AEA13E042E050E0B801CE01B7
:1039D0008F579F4F0E94792A40E850E0BE016F5FE9
:1039E0007F4FCF57DF4F88819981C158D0400E94C7
:1039F0003D1B882379F00E5F1F4F93E0063B1907AC
:103A000019F781E08093DA030E94FC229093E3038C
:103A10008093E2038091DA03CE57DF4F0FB6F8941C
:103A2000DEBF0FBECDBFDF91CF911F910F910895E3
:103A3000CF93DF93CDB7DEB7E0970FB6F894DEBF34
:103A40000FBECDBF8091DA03811105C00E94B11C69
:103A5000882309F46DC081E00E94EF198AE090E0AC
:103A60000E947D1B8091E2039091E3030E94142346
:103A7000893E9340C8F18091DB03811117C040E378
:103A800050E0BE016F5F7F4F8AE393E00E943D1BD1
:103A9000882349F040E350E0BE016F5F7F4F87E22B
:103AA00093E00E943D1B81E08093DB030E94FC2297
:103AB0009093E3038093E20340E350E0BE016F5F25
:103AC0007F4F89E193E00E943D1B882369F0CE017E
:103AD00001960E945B2A21E0892B09F420E0809165
:103AE000D80382132093D8038091DC039091DD03E7
:103AF0000E94142381319742D8F090914402809122
:103B00004502981315C00E94FC229093DD03809318
:103B1000DC0385E30E945419092E000CAA0BBB0B91
:103B20008093DE039093DF03A093E003B093E1035F
:103B3000E0960FB6F894DEBF0FBECDBFDF91CF91F8
:103B400008950F931F93CF93DF93EC01FB018C013A
:103B500000571E4FD8012C9130E0C901019668E250
:103B600070E00E942D2ADE01AF56BE4F9C9198173F
:103B700081F09AE0929FD001939FB00D1124AC0F79
:103B8000BD1F01900D929A95E1F7F801808381E0C5
:103B900001C080E0DF91CF911F910F910895FF92B6
:103BA0000F931F93CF93DF93CDB7DEB72A970FB64E
:103BB000F894DEBF0FBECDBF8B01F42E19828C832B
:103BC0000E94FC229B838A83F80180818D83FF20E1
:103BD00011F0818101C080E08E83F1E0FF1518F4BF
:103BE000F801828101C080E08F83F2E0FF1518F4B4
:103BF000F801838101C080E08887F3E0FF1518F4A5
:103C0000F801848101C080E08987F4E0FF1518F491
:103C1000F801858101C080E08A87BE016F5F7F4F18
:103C200086E492E00E94A11D811105C086E990E022
:103C30000E947D1BC9CFF6E0FF1528F48AEFF80E2D
:103C40000A5F1F4FC1CF2A960FB6F894DEBF0FBE92
:103C5000CDBFDF91CF911F910F91FF900895CF932A
:103C6000DF93CDB7DEB72A970FB6F894DEBF0FBE4D
:103C7000CDBF21E029839D838C83BE016F5F7F4F81
:103C800086E492E00E94A11D811105C086E990E0C2
:103C90000E947D1BF2CF2A960FB6F894DEBF0FBEAE
:103CA000CDBFDF91CF9108950F93CF93DF93CDB721
:103CB000DEB72A970FB6F894DEBF0FBECDBF92E0F5
:103CC00099838C836D834E832F830887BE016F5F3A
:103CD0007F4F86E492E00E94A11D811105C086E914
:103CE00090E00E947D1BF2CF2A960FB6F894DEBFBB
:103CF0000FBECDBFDF91CF910F9108951092D603E3
:103D00001092D703E0E4F2E014821582089589321C
:103D100089F1F0F4843171F1B0F4873009F077C0A3
:103D200081E080930B0184E180930A018AE0809313
:103D300009018EE18093080188E08093050188E203
:103D40008093040164C092EE980F9A30F0F05FC047
:103D5000803509F444C028F48F3409F058C08AE053
:103D60003FC0813529F0823509F051C081E038C06B
:103D70008FEF36C08091E603882379F11092E60335
:103D80001092E5031092E40342C08D518093E60344
:103D9000833099F038F4813069F08230D9F48AE0C8
:103DA00091E00DC0853099F078F0863099F484E088
:103DB00091E005C08BE091E002C089E091E0909332
:103DC000E5038093E40323C088E091E0F8CF85E029
:103DD00091E0F5CF1092E6031AC080E0089586EFD7
:103DE000E091E403F091E503309789F02081082EFB
:103DF000000C990B820F911D8F3F910519F014F063
:103E00008FEF04C097FF02C0108201C0808381E061
:103E100008950F931F9341E050E060E070E08A0145
:103E20009B0104C0000F111F221F331F8A95D2F778
:103E3000C901B8010E9410091F910F910C94B80894
:103E40008B3109F468C058F58B3009F486C078F4DA
:103E5000863009F445C020F4853009F44BC07FC09A
:103E6000873009F44AC0883009F477C078C08031BF
:103E700009F464C068F48E3009F071C080912E029C
:103E800082FB222720F991E0922790FB82F94CC017
:103E9000863109F462C0893109F45FC060C08A329A
:103EA000E1F060F4873209F455C028F48E3108F44B
:103EB00056C08D5150C08932E9F051C0833450F45E
:103EC0008A3308F045C0853309F444C0883309F4C7
:103ED00044C045C08334F1F142C00E94990F3DC0F7
:103EE00080912E02817F8E7F80932E0281E08093CD
:103EF000E70308950E94700330C080912E02982F2E
:103F00009095917090FB80F980932E02911125C0BD
:103F1000897F877F10C080912E0281FB222720F9A4
:103F200091E0922790FB81F980932E029923A9F0CA
:103F300080912E02816080932E020FC080912E020C
:103F400083FB222720F991E0922790FB83F9ECCFA5
:103F5000895301C080E00E94091F81E0089580E03C
:103F6000089580E008950C94B11FCF93C82F8091DD
:103F7000E703813069F038F08230C1F58C2F0E9460
:103F8000871E81E039C00E940B0E823289F504C081
:103F90000E940B0E823261F48C2F0E94B31F81119C
:103FA00004C08C2F0E94201F1FC081E090E01CC025
:103FB0008C2F0E94B11F811116C0C43189F058F4B2
:103FC000CB3089F0C031B1F482E08093E70388E31D
:103FD0000E94871E08C0C93219F0C83321F00AC0F8
:103FE0001092E70307C081E0817006C01092E703DA
:103FF00080E002C080E0F8CFCF910895CF93DF93A7
:1040000086319C4541F5EB010E940B0E982F8A8169
:104010002091020130910301882379F09A7A81E09E
:1040200009F480E08093E803911102C069E201C0C5
:1040300065E3C9010E949D220AC08091E8038111B5
:1040400002C069E201C065E3C9010E949F220E948B
:10405000500E80E001C081E0DF91CF9108950F9371
:104060001F93CF93DF93C42FD22FFC01828188232B
:10407000C9F04093EB030E94FC229093EA038093E3
:10408000E90380E28C0F883008F057C0C77081E0E8
:1040900001C0880FCA95EAF7DF91CF911F910F9168
:1040A0000C9407068091EB03481330C08091E9031C
:1040B0009091EA030E941423883C910538F510E2A0
:1040C0001D0FCD17B9F080E28C0F883040F4C77017
:1040D00081E001C0880FCA95EAF70E940E061830E9
:1040E00028F581E09D2F977001C0880F9A95EAF717
:1040F0000E940706802F0E94FE051830F0F4D7704A
:1041000081E001C0880FDA95EAF70AC080E28C0FDF
:10411000883098F4C77081E001C0880FCA95EAF72B
:10412000DF91CF911F910F910C940E06802FDF919C
:10413000CF911F910F910C94FE05DF91CF911F91AC
:104140000F9108950F939C01CB01243F4CE5340758
:1041500031F188F4293DFCE53F07D9F02A3D4CE5D3
:10416000340779F1283D3C45A9F506E221EE41EE00
:1041700068ED7CE52BC0263FFCE53F07E1F0A8F0A9
:10418000273F3C4539F507E225EE46EE67EF7CE533
:104190001DC007E225EE45EE69ED7CE517C006E29D
:1041A00021EE40EE64EF7CE511C007E225EE44EE1F
:1041B00065EF7CE50BC006E221EE42EE66EF7CE5A2
:1041C00005C008E221E045EE6AED7CE50E942F2063
:1041D00080E008C0FC018281882319F01092EB0373
:1041E00001C081E00F910895289A219A229A23987C
:1041F0002B9880E58CBD089590910D019F3F09F0AB
:1042000072C08F3F09F46FC0611103C01092ED03BB
:1042100003C090E29093ED03423041F0433051F0FF
:10422000413069F49091ED03946007C09091ED03E3
:10423000986003C09091ED039C609093ED0341E082
:1042400050E04217530718F4440F551FFACF9091CE
:10425000ED0340315105F1F050F442305105B1F019
:1042600048305105E1F421E02093EC0313C04034C1
:10427000510591F04038510539F04032510579F43B
:1042800021E02093EC0308C0936007C091E0909375
:10429000EC0305C0916001C092609093ED032CB5D2
:1042A0009091ED03922B9CBD9091EC03992319F012
:1042B0009DB591609DBD80930D01E82FE295EF7053
:1042C000F0E031A1282F2F7081E090E001C0880F2D
:1042D0002A95EAF7932F982B91A392A18095892391
:1042E00082A381E0089580E00895CF93DF938EBD8F
:1042F0000E94FC22EC010DB407FC0AC00E94FC22C3
:104300008C1B9D0B84369105B0F38EEF9FEF02C09E
:104310008EB590E0DF91CF910895CF93DF931EBCCF
:104320000E94FC22EC010DB407FC0AC00E94FC2292
:104330008C1B9D0B84369105B0F38EEF9FEF02C06E
:104340008EB590E0DF91CF9108950F931F93CF9397
:10435000DF93EC018C01060F171FC017D10731F056
:1043600089910E94752197FD03C0F7CF80E090E00E
:10437000DF91CF911F910F9108950F931F93CF93CA
:10438000DF93EC018C01060F171FC017D10731F026
:104390000E948D2197FD04C08993F7CF80E090E0C3
:1043A000DF91CF911F910F91089580910D018F3F63
:1043B00019F1E82FE295EF70F0E031A1282F2F706E
:1043C00081E090E001C0880F2A95EAF7932F982B9F
:1043D00091A392A1892B82A38FEF80930D018DB5BC
:1043E0008E7F8DBD9CB58091ED03809589238CBD1A
:1043F0001092ED031092EC0308959093A90180931D
:10440000A80108959093F3038093F2030895E09137
:10441000F203F091F303309721F00190F081E02D49
:10442000099480E008950E9407220895E091F20324
:10443000F091F303309721F00280F381E02D09948D
:104440000895E091F203F091F303309739F022E000
:10445000DC012C930480F581E02D099408952091CE
:10446000F0033091F1032817390771F09093F103AD
:104470008093F003E091F203F091F303309721F081
:104480000680F781E02D099408952091EE03309184
:10449000EF032817390771F09093EF038093EE0331
:1044A000E091F203F091F303309721F00084F1855D
:1044B000E02D09940895FC01329697E080E0915038
:1044C00029F021912223D9F38F5FF9CF0895662334
:1044D00049F0FC01329608962191621729F0E817FD
:1044E000F907D1F780E0089581E008959C01FC016F
:1044F00032969FEF80E04191461789F09F3F19F473
:10450000411101C0982F8F5F8630A9F79F3F39F086
:10451000F901E90FF11D97FDFA9562830895089559
:104520009C012A5F3F4FFC014281461301C0128269
:10453000019682179307B9F708950C9476220C948C
:104540009022029626E0FC0111922A95E9F708953F
:1045500008950C94A82283E08093F4030C94A9227C
:10456000811102C081E001C082E08093F4030C94C9
:10457000A9220C94B02281E08093F4030C94A92228
:104580000C94BB2208950C94C22208951F920F929E
:104590000FB60F9211248F939F93AF93BF93809187
:1045A000F503811113C080911C0490911D04A0910A
:1045B0001E04B0911F044196A11DB11D80931C04DF
:1045C00090931D04A0931E04B0931F04BF91AF915C
:1045D0009F918F910F900FBE0F901F9018950E9482
:1045E000B8080C94EC0382E084BD93E095BD9DE790
:1045F00097BD80936E0008952FB7F89480911C04A6
:1046000090911D04A0911E04B0911F042FBF089526
:104610002FB7F89460911C0470911D0480911E04C2
:1046200090911F042FBF08959C014FB7F89480917B
:104630001C0490911D04A0911E04B0911F044FBF53
:10464000821B930B089578941F920F920FB60F92CE
:1046500011248F939F93AF93BF9380911C049091EB
:104660001D04A0911E04B0911F040196A11DB11D4F
:1046700080931C0490931D04A0931E04B0931F0408
:10468000BF91AF919F918F910F900FBE0F901F9090
:10469000189587E797E790930108809300089AE0C0
:1046A00088E10FB6F894A895809360000FBE9093B0
:1046B0006000FFCF80910104089508950F93CF9378
:1046C000DF93EC010E94F618833041F409812D81BB
:1046D0004C816B818A810E94541E1FC082E08093AE
:1046E000E9008FEF9091E800815095FD06C09AE6B1
:1046F0009A95F1F700C08111F5CF8091E80085FF10
:104700000CC040E050E066E070E0CE010E948C25D5
:104710008091E8008E778093E800DF91CF910F9130
:104720000895CF93DF93EC010E94F618833049F48B
:10473000BE016E5F7F4F46E08881DF91CF910C9480
:10474000CF1D81E08093E9008FEF9091E8008150C8
:1047500095FD06C09AE69A95F1F700C08111F5CF54
:104760008091E80085FF14C040E050E068E070E010
:10477000CE010E948C258091E8008E778093E8001E
:1047800088E0FE01A9EFB3E001900D928A95E1F770
:10479000DF91CF9108958093F6037093F8036093AF
:1047A000F70380912404843001F582E08093E900CE
:1047B0008FEF9091E800815095FD06C09AE69A959A
:1047C000F1F700C08111F5CF8091E80085FF0DC0A1
:1047D00040E050E063E070E086EF93E00E948C25BB
:1047E0008091E8008E778093E8000895CF93DF935F
:1047F000EC010E94F618833029F4CE01DF91CF91AD
:104800000C942F1EBE0184E0DF91CF910C94CB233A
:10481000BC0183E00C94CB2380912304811109C057
:104820000E941D270E947A278091E2008460809375
:10483000E20008951092230408950C94C022609120
:10484000200481E0611101C080E00C94AB220E9441
:10485000EF229091240481E0943009F080E060918F
:1048600020040C94B02242E061EC81E00E94962684
:1048700042E261EC82E00E9496269091240481E05D
:10488000943009F080E0609120040C94B92280916A
:104890002604833009F461C030F4813071F0823035
:1048A00009F49AC008958A3009F486C08B3009F45F
:1048B0006CC0893009F0A8C020C080912504813ADD
:1048C00009F0A2C08091E800877F8093E800809182
:1048D000290490912A04892B21F468E089EF93E060
:1048E00003C060E080E090E070E00E94D7258091F6
:1048F000E8008B778093E800089580912504813249
:1049000009F082C08091290490912A04029708F04E
:104910007BC08091E800877F8093E8008091E80069
:1049200082FD05C0809124048111F8CF6DC02091D3
:10493000F3008091F20090E0922B029731F4809185
:10494000F100813011F0863021F48091F1008093E4
:1049500001048091E8008B7753C080912504813A4F
:1049600009F052C08091290490912A04892B09F002
:104970004BC08091E800877F8093E8008091E80039
:1049800080FFFCCF80911A0136C0809125048132CE
:10499000D9F58091290490912A04892BA9F5809159
:1049A000E800877F8093E8000E94CB26809127044F
:1049B00080931A010C94B80880912504813221F566
:1049C0008091E800877F8093E8000E94CB26809149
:1049D000280480930204089580912504813AA1F46B
:1049E0008091E800877F8093E8008091E80080FF55
:1049F000FCCF809102048093F1008091E8008E77D3
:104A00008093E8000C94CB26089584B7877F84BFF9
:104A10000FB6F894A895809160008861809360003B
:104A2000109260000FBE90E080E80FB6F89480937B
:104A30006100909361000FBE0C94BB220E941D2761
:104A40000E947A27E2EEF0E080818460808378948F
:104A50000C940C2A8EE091E00C94022208950C94A0
:104A6000181D0C943325292F332723303105C9F025
:104A700060F42130310581F02230310509F044C065
:104A80008BE390E024EE33E043C021323105E1F0C6
:104A90002232310549F138C082E190E02FE134E063
:104AA00037C099278130910549F028F0029761F5C8
:104AB000E6EBF3E005C0E0EEF3E002C0E6ECF3E085
:104AC000849190E09F0124C06115710541F061302F
:104AD0007105D1F489E090E02FE034E019C089E05D
:104AE00090E026EF33E014C06115710541F06130AC
:104AF000710551F48BE790E021E334E009C080E4D4
:104B000090E02CEA34E004C080E090E020E030E067
:104B1000FA01318320830895CF92DF92EF92FF92C2
:104B20000F931F93CF93DF93EC018B017A010E94C7
:104B3000EA26811133C0E114F10439F0F7018081D4
:104B40009181081B190BC80FD91FC12CD12C01153D
:104B5000110519F18091E80085FD16C08091E800EB
:104B60008E778093E800E114F10449F0F701808129
:104B70009181C80ED91ED182C08285E00FC00E94EB
:104B8000EA26882321F30AC089918093F10001501D
:104B90001109FFEFCF1ADF0ADACF80E0DF91CF9162
:104BA0001F910F91FF90EF90DF90CF90089520918B
:104BB0002B0430912C042617370748F06115710536
:104BC00039F42091E8002E772093E80001C0B90164
:104BD000FC0120E06115710579F18091240488239E
:104BE000F1F18530F1F18091E80083FD3CC08091C6
:104BF000E80082FD2EC08091E80080FFEBCF20917D
:104C0000F3008091F20090E0922B6115710551F054
:104C10008830910538F421912093F1006150710999
:104C20000196F3CF21E0089709F020E08091E80099
:104C30008E778093E800CECF2111CFCF0AC080912C
:104C40002404882361F0853061F08091E80083FDC1
:104C50000AC08091E80082FFF2CF80E0089582E0F0
:104C6000089583E0089581E0089520912B04309108
:104C70002C042617370748F06115710539F4209187
:104C8000E8002E772093E80001C0B901FC0120E084
:104C90006115710591F180912404882309F440C0C5
:104CA000853009F43FC08091E80083FD3DC08091CC
:104CB000E80082FD2FC08091E80080FFE9CF2091BD
:104CC000F3008091F20090E0922B6115710559F08C
:104CD0008830910540F424912093F1003196615081
:104CE00071090196F2CF21E0089709F020E0809148
:104CF000E8008E778093E800CBCF2111CCCF0AC09B
:104D000080912404882361F0853061F08091E8006F
:104D100083FD0AC08091E80082FFF2CF80E0089511
:104D200082E0089583E0089581E00895982F9730F8
:104D300068F59093E900981739F07091EC00209194
:104D4000ED005091F00003C0242F762F50E021FD9C
:104D500002C09F5FECCF3091EB003E7F3093EB00C1
:104D60003091ED003D7F3093ED003091EB003160EC
:104D70003093EB007093EC002093ED005093F00023
:104D80002091EE0027FDE5CF80E008958F7080939D
:104D9000E90081E008958091250487FF11C080918A
:104DA000E80082FD05C0809124048111F8CF11C074
:104DB0008091E8008B770BC080912404882349F010
:104DC0008091E80080FFF8CF8091E8008E77809393
:104DD000E80008952091E4003091E50095E64091C7
:104DE000EC00842F817040FF23C08091E80080FD9B
:104DF0001DC080912404882399F0853099F080911A
:104E0000EB0085FD11C04091E4005091E5002417AE
:104E1000350729F3915011F09A01E1CF84E008950C
:104E200082E0089583E0089581E0089580E0089588
:104E30004091E80042FFDDCF08950E948B270E9439
:104E40009327E0EEF0E0808181608083E8EDF0E080
:104E500080818F77808319BCA7EDB0E08C918E7F25
:104E60008C9380818F7E80831092230408950F930A
:104E70001F93CF93DF930E948B270E949327C8ED47
:104E8000D0E088818F778883888180688883888153
:104E90008F7D888319BC10922404109220041092F4
:104EA00022041092210400EE10E0F80180818B7F33
:104EB000808388818160888342E060E080E00E9496
:104EC0009626E1EEF0E080818E7F8083E2EEF0E0D6
:104ED000808181608083808188608083F801808107
:104EE0008E7F8083888180618883DF91CF911F913D
:104EF0000F910895E8EDF0E080818F7E8083E7EDEB
:104F0000F0E080818160808384E082BF81E08093D3
:104F100023040C943727E8EDF0E080818E7F8083B6
:104F20001092E20008951092DA001092E1000895C4
:104F30001F920F920FB60F9211242F933F934F930E
:104F40005F936F937F938F939F93AF93BF93EF93F1
:104F5000FF938091E10082FF0BC08091E20082FF0D
:104F600007C08091E1008B7F8093E1000E940B2AB3
:104F70008091DA0080FF1DC08091D80080FF19C0A9
:104F80008091DA008E7F8093DA008091D90019BC7D
:104F900080FF0BC082E089BD09B400FEFDCF81E037
:104FA000809324040E940C2404C0109224040E94C4
:104FB0001A248091E10080FF19C08091E20080FFF7
:104FC00015C08091E2008E7F8093E2008091E20024
:104FD00080618093E2008091D80080628093D80045
:104FE00019BC85E0809324040E941F248091E10075
:104FF00084FF2FC08091E20084FF2BC019BC82E0A7
:1050000089BD09B400FEFDCF8091D8008F7D8093CB
:10501000D8008091E1008F7E8093E1008091E200D2
:105020008F7E8093E2008091E20081608093E200B5
:1050300080912004882311F084E007C08091E30070
:1050400087FD02C081E001C083E0809324040E94B8
:1050500027248091E10083FF29C08091E20083FF33
:1050600025C08091E100877F8093E10082E08093FA
:105070002404109220048091E1008E7F8093E1004F
:105080008091E2008E7F8093E2008091E200806157
:105090008093E20042E060E080E00E9496268091EA
:1050A000F00088608093F0000E941D24FF91EF9132
:1050B000BF91AF919F918F917F916F915F914F9130
:1050C0003F912F910F900FBE0F901F9018951F9238
:1050D0000F920FB60F9211242F933F934F935F932C
:1050E0006F937F938F939F93AF93BF93CF93DF93F0
:1050F000EF93FF93C091E900CF708091EC00D82F1F
:10510000D17080FDD0E81092E9008091F000877F97
:105110008093F00078940E94AB281092E90080916F
:10512000F00088608093F000CD2BCF70C093E90031
:10513000FF91EF91DF91CF91BF91AF919F918F91AF
:105140007F916F915F914F913F912F910F900FBE83
:105150000F901F9018951F93CF93DF93CDB7DEB7B5
:10516000AA970FB6F894DEBF0FBECDBFE5E2F4E01C
:105170008091F100819324E0ED32F207C9F70E949B
:1051800047248091E80083FF2EC1809125049091EF
:105190002604492F50E04A30510508F024C1FA0195
:1051A000EE59FF4F0C94412A803821F0823809F0E3
:1051B0001AC108C08091210490912204992389F09A
:1051C00082600FC0809129048F70873008F00BC176
:1051D0008093E9008091EB0085FB882780F910928D
:1051E000E9009091E800977F9093E8008093F100A8
:1051F0001092F100D1C0282F2D7F09F0F4C0882330
:1052000019F0823061F0EFC080912704813009F0FD
:10521000EAC0933009F080E0809322042EC0809190
:10522000270481112AC0809129048F702FEF280F45
:10523000263008F0D8C08093E9002091EB0020FFD1
:105240001CC0933021F48091EB00806214C09091D7
:10525000EB0090619093EB0021E030E0A90102C0E7
:10526000440F551F8A95E2F74093EA001092EA0036
:105270008091EB0088608093EB001092E9008091B0
:10528000E800877F8093E8000E94CB26ACC08111A4
:10529000AAC0109127041F778091E3008078812BAA
:1052A0008093E3008091E800877F8093E8000E946C
:1052B000CB268091E80080FFFCCF8091E3008068DE
:1052C0008093E300111102C082E001C083E080936B
:1052D000240489C08058823008F085C0809127045A
:1052E000909128048C3D53E0950779F583E08A83FB
:1052F0008AE289834FB7F894DE01139620E03EE0FE
:1053000051E2E32FF0E050935700E49120FF03C0F7
:10531000E295EF703F5FEF708E2F90E0EA3010F073
:10532000C79601C0C0968D939D932F5F243149F796
:105330004FBF8091E800877F8093E8006AE270E0C9
:10534000CE0101960E94D72516C060912904709164
:105350002A04AE014F5F5F4F0E943125BC01892BAB
:1053600009F441C09091E800977F9093E80089810B
:105370009A810E9435268091E8008B778093E8001F
:1053800032C0803881F58091E800877F8093E80003
:10539000809120048093F1008091E8008E7772CF95
:1053A000811121C0809127049091280499270297A8
:1053B000D4F48091E800877F8093E80080912704EF
:1053C000809320040E94CB2680912004811106C086
:1053D0008091E30087FD02C081E001C084E08093FA
:1053E00024040E9433248091E80083FF0AC0809146
:1053F000E800877F8093E8008091EB0080628093D3
:10540000EB00AA960FB6F894DEBF0FBECDBFDF91BA
:10541000CF911F9108950895CF93809124048823FC
:10542000A1F0C091E900CF709091EC00892F8170BC
:1054300090FD80E8C82B1092E9008091E80083FD80
:105440000E94AB28CF70C093E900CF91089580915E
:10545000E300881F8827881F089597FB072E16F4FE
:10546000009407D077FD09D00E94472A07FC05D099
:105470003EF4909581959F4F0895709561957F4F6B
:105480000895EE0FFF1F0590F491E02D0994AA1BDB
:10549000BB1B51E107C0AA1FBB1FA617B70710F01F
:1054A000A61BB70B881F991F5A95A9F78095909551
:1054B000BC01CD010895FC0188279927E89421912A
:1054C0002032E9F3293010F02E30C8F32B3241F0AE
:1054D0002D3239F4689404C00E94C72A820F911DAE
:1054E000219120532A30C0F31EF4909581959F4F4F
:1054F0000895FB01DC0102C005900D92415050401F
:10550000D8F70895FB01DC018D91059080190110F9
:10551000D9F3990B0895FB01DC0105900D92002051
:10552000E1F70895FC0105900020E9F7809590953A
:105530008E0F9F1F0895FB01DC0104C08D91019027
:10554000801921F441505040C8F7881B990B0895E9
:10555000FB01DC0102C001900D9241505040D8F790
:105560000895FB01DC010D900020E9F711970190EF
:105570000D920020E1F70895FC0181E090E0019098
:10558000061609F4CF010020D1F7019708957AE0BB
:10559000979F902D879F802D910D11240895AEE047
:1055A000B0E0E5EDFAE20C94E02D0D891E898F89BB
:1055B000988D26E02C831A83098397FF02C080E030
:1055C00090E801979E838D83AE01455E5F4F698DA4
:1055D0007A8DCE0101960E94FF2A4D815E8157FD92
:1055E0000AC02F813885421753070CF49A01F8013D
:1055F000E20FF31F10822E96E4E00C94FC2DABE03A
:10560000B0E0E5E0FBE20C94D22D6C017B018A0155
:10561000FC0117821682838181FFCCC1CE010196E5
:105620003C01F6019381F70193FD859193FF8191F0
:105630007F01882309F4BAC1853239F493FD85913D
:1056400093FF81917F01853229F4B60190E00E9499
:10565000F62CE7CF912C212C312CFFE1F315D8F05B
:105660008B3279F038F4803279F08332A1F4232D33
:1056700020611DC08D3261F0803369F4232D2160DB
:1056800016C0832D8260382EE32DE4603E2E2AC0A2
:10569000F32DF8601DC037FC2DC020ED280F2A30F7
:1056A00040F08E32B9F436FC81C1232D2064322EB5
:1056B00019C036FE06C08AE0989E200D1124922E55
:1056C00011C0EAE02E9E200D1124222EF32DF0624F
:1056D0003F2E08C08C3621F4832D8068382E02C0FE
:1056E000883641F4F70193FD859193FF81917F0105
:1056F0008111B3CF982F9F7D9554933028F40C5F80
:105700001F4F9FE399830DC0833631F0833771F0CB
:10571000833509F059C021C0F801808189830E5F6B
:105720001F4F88248394912C530113C02801F2E069
:105730004F0E511CF801A080B18036FE03C0692DC8
:1057400070E002C06FEF7FEFC5010E94EB2C4C01AF
:105750008201F32DFF773F2E16C0280122E0420E72
:10576000511CF801A080B18036FE03C0692D70E0A5
:1057700002C06FEF7FEFC5010E94E02C4C01F32DBA
:10578000F0683F2E820133FC1BC0822D90E088160A
:105790009906B0F4B60180E290E00E94F62C2A94BB
:1057A000F4CFF50137FC859137FE81915F01B60199
:1057B00090E00E94F62C21102A9421E0821A910890
:1057C0008114910471F7E8C0843611F0893641F5EF
:1057D000F80137FE07C060817181828193810C5F7F
:1057E0001F4F08C060817181072E000C880B990B38
:1057F0000E5F1F4FF32DFF763F2E97FF09C0909548
:105800008095709561957F4F8F4F9F4FF0683F2E29
:105810002AE030E0A3010E94322D882E861845C070
:10582000853731F4232D2F7EB22E2AE030E025C0BB
:10583000932D997FB92E8F36C1F018F4883579F001
:10584000B5C0803719F0883721F0B0C0E92FE0618A
:10585000BE2EB4FE0DC0FB2DF460BF2E09C034FE79
:105860000AC0292F2660B22E06C028E030E005C00D
:1058700020E130E002C020E132E0F801B7FE07C0CD
:1058800060817181828193810C5F1F4F06C06081AE
:10589000718180E090E00E5F1F4FA3010E94322DC6
:1058A000882E8618FB2DFF773F2E36FE0DC0232D48
:1058B0002E7FA22E891458F434FE0BC032FC09C08E
:1058C000832D8E7EA82E05C0B82CA32C03C0B82C27
:1058D00001C0B92CA4FE0FC0FE01E80DF11D8081AE
:1058E000803321F49A2D997EA92E09C0A2FE06C00C
:1058F000B394B39404C08A2D867809F0B394A3FCC2
:1059000011C0A0FE06C0B21488F4280C922C9B187B
:105910000EC0B21460F4B60180E290E00E94F62C52
:10592000B394F7CFB21418F42B1802C0982C212C82
:10593000A4FE10C0B60180E390E00E94F62CA2FE07
:1059400017C0A1FC03C088E790E002C088E590E0A2
:10595000B6010CC08A2D867859F0A1FE02C08BE2F8
:1059600001C080E2A7FC8DE2B60190E00E94F62C17
:10597000891438F4B60180E390E00E94F62C9A94E2
:10598000F7CF8A94F301E80DF11D8081B60190E014
:105990000E94F62C8110F5CF222009F442CEB601E8
:1059A00080E290E00E94F62C2A94F6CFF6018681E0
:1059B000978102C08FEF9FEF2B96E2E10C94EE2DC2
:1059C000FC010590615070400110D8F780959095CA
:1059D0008E0F9F1F0895FC016150704001900110CF
:1059E000D8F7809590958E0F9F1F08950F931F9362
:1059F000CF93DF93FB01238121FD03C08FEF9FEF46
:105A00002CC022FF16C04681578124813581421760
:105A1000530744F4A081B1819D012F5F3F4F318333
:105A200020838C93268137812F5F3F4F37832683D6
:105A300014C08B01EC01FB010084F185E02D099578
:105A4000892BE1F6D80116968D919C9117970196B6
:105A500017969C938E931697CE01DF91CF911F914D
:105A60000F910895FA01AA27283051F1203181F1D0
:105A7000E8946F936E7F6E5F7F4F8F4F9F4FAF4F56
:105A8000B1E03ED0B4E03CD0670F781F891F9A1F69
:105A9000A11D680F791F8A1F911DA11D6A0F711D1D
:105AA000811D911DA11D20D009F468943F912AE029
:105AB000269F11243019305D3193DEF6CF01089511
:105AC000462F4770405D4193B3E00FD0C9F7F6CF42
:105AD000462F4F70405D4A3318F0495D31FD40520A
:105AE000419302D0A9F7EACFB4E0A69597958795A0
:105AF00077956795BA95C9F700976105710508957F
:105B00009B01AC010A2E069457954795379527952A
:105B1000BA95C9F7620F731F841F951FA01D0895C2
:105B2000F999FECF92BD81BDF89A992780B5089565
:105B3000A8E1B0E042E050E00C94C42D262FF99982
:105B4000FECF92BD81BDF89A019700B4021639F0DC
:105B50001FBA20BD0FB6F894FA9AF99A0FBE0895AD
:105B60000396272F0E949F2D0E949E2D252F0E9475
:105B70009F2D242F0C949F2D0196272F0E949F2D3F
:105B80000C949E2DDC01CB01FC01F999FECF06C0DF
:105B9000F2BDE1BDF89A319600B40D9241505040EB
:105BA000B8F708952F923F924F925F926F927F9233
:105BB0008F929F92AF92BF92CF92DF92EF92FF921D
:105BC0000F931F93CF93DF93CDB7DEB7CA1BDB0BC9
:105BD0000FB6F894DEBF0FBECDBF09942A8839886E
:105BE00048885F846E847D848C849B84AA84B98475
:105BF000C884DF80EE80FD800C811B81AA81B98181
:105C0000CE0FD11D0FB6F894DEBF0FBECDBFED0194
:065C10000895F894FFCF97
:105C1600C8001402280850011E0A140140FF5A2326
:105C260091235E230824F6235D2301E200E900EABE
:105C360000B500B600B700CD008301CC008A019202
:105C46000194012102230224022502260227022AA8
:105C560002B300B4006F007000818283E200E900A5
:105C6600EA00B500B600B700CD008301CC008A017A
:105C76009201940121022302240225022602270210
:105C86002A02B300B4006F007000818283973591B9
:105C9600906636F09293F4F1379667F54C00520011
:105CA6004D00300041542B424C45504F5745524C05
:085CB6004556454C3D256400F4
:00000001FF
